:020000003628A0
:08000800A000030E8301A1001A
:100010000408A2000C1C2F280C1023085820A40050
:10002000A5012418A515A41825162419A516A41988
:100030002515241AA514A41A251425088700A5013E
:10004000241B2515A41BA51625088500A30A10301E
:1000500023020319A301AA308E00F0308F0022087A
:100060008400210E8300A00E200E090085010130BE
:100070008316850083128701831687018312A030BF
:100080008700A3018B170B170C10101483160C1488
:100090008312AA308E00FF308F004D288207003473
:1000A0000034FF34813481348134FF34003400342F
:1000B00082070034FF3489348934813400340034B9
:1000C0003C344234813481344234003400340034CE
:0200D0000034FA
:02400E00D43F9D
:00000001FF
